:020000020000FC
:100000005AC937C20000000023C000004FC10000E1
:10001000000052C1000000000000000002030406BE
:10002000080C101820304060800002030406080C01
:10003000101820304080FF000406080C10182030F3
:10004000406080A0C00005050D050D0603030302F6
:100050004FB662FD20C070FF1CC165FDFCC057FE9D
:1000600001C00994C0919700C395C0939700C5E063
:10007000C519B8F3D0919700CD1B98F3C8E7089441
:1000800083FDC795C4BDC52DCC2321F4C0E083FDFD
:10009000C0E8C4BD09C171FF03C0919890989398BE
:1000A000C52D089483FDC795C4BDC09399006B7F8F
:1000B000C52DCF3F09F443C0C0919800C395C093AC
:1000C000980070FF37C082FD05C091989098939872
:1000D0004FBE18957860C091A000CC2391F0C091DC
:1000E0009800CA95D091A000CD1B58F0777FC091A1
:1000F0009800D0919F00CD1B08F41CC0209298005E
:1001000019C0919890989398C5E0CA95F1F7C0915D
:100110007500CA95C2FD09C0C1FD05C095FF95983F
:1001200095FD94980EC097980CC095FF949895FDF6
:10013000959807C09198909893984FBE18952092E3
:1001400099004FBE1895A5C0552021F095FF919AB2
:1001500095FD939A90989DC0552009F0909A95FF2F
:10016000939895FD919895C0552021F095FF939A0D
:1001700095FD919A95FF919895FD93988AC095FF6A
:10018000949A95FD959A95FF959A95FD949AC5E058
:10019000CA95F1F7552021F095FF919A95FD939A14
:1001A000909877C095FF949A95FD959A979AC5E097
:1001B000CA95F1F7552021F095FF919A95FD939AF4
:1001C000909867C0979A95FF949A95FD959AC5E087
:1001D000CA95F1F7552009F0909A95FF939895FDEF
:1001E000919857C0979A95FF959A95FD949AC5E076
:1001F000CA95F1F7552009F0909A95FF939895FDCF
:10020000919847C095FF959A95FD949A979AC5E065
:10021000CA95F1F7552021F095FF939A95FD919A93
:1002200095FF919895FD939834C095FF959A95FD0B
:10023000949A95FF949A95FD959AC5E0CA95F1F721
:10024000552021F095FF939A95FD919A95FF9198ED
:1002500095FD93981EC082FF1CC0C0917500C2FD21
:100260000BC0C1FD11C095FF949A95FD959A95FF1D
:10027000959A95FD949A0DC0C1FDF5CF95FF949A7E
:1002800095FD959A979A05C0979A95FF959A95FD31
:10029000949AC52DC095089483FDC795C4BDC0939D
:1002A00099002092970064604FBE18954FB6C0E148
:1002B000C8BF6E7F4FBE18953FB68F7EABB7A07498
:1002C000A2118061A0E0ABBFA9B7AE7FA9BF7894AF
:1002D000A0916600AA2349F0A92FAF7151F1A09116
:1002E0006600AA95A093660024C040E050E0A0B349
:1002F00096FDA095A2FD4FEF96FFA3E096FDA2E02C
:10030000A5BFAA27A064AABF8D7FA0B396FDA09524
:10031000A2FD5FEF451749F7A8E161FDA0936600D4
:10032000A92FAF7119F0A8E1A093660040938D004A
:100330008160A0916700AA2331F0A0916700AA957F
:10034000A093670007C0A92FAF7121F08061AA2791
:10035000A064AABF80FF48C0A0918D004A2F8E7F65
:10036000A92FAF71C1F0403F08F040EFA42FA29534
:10037000AF704A0F5091B000533069F0A695A69522
:1003800050FD01C0A69552FD03C0A41B4A2F03C017
:100390004A0F08F44FEFA09196004A1708F44A2F2D
:1003A0004093610071FF08C0A091610050919200DC
:1003B000A51710F050936100A09161004091630077
:1003C000A41B70F04091CF00A40B50F0A0916300EB
:1003D000A40FA093630040F4AFEFA093630004C0A8
:1003E000A0916100A093630040916300A0919200EE
:1003F0004A1708F04A2F542EA52DA03408F0686043
:10040000A0916000A395A093600051F0F894A9B763
:10041000A160A9BF84FF02C0A0E4ABBF3FBE189596
:1004200041E050916600552331F0A92FAF7119F4C6
:100430005A9550936600A0918D00A13018F020923B
:1004400090000DC02092910020929A00A0919000FF
:10045000AF5FA093900018F0AFEFA0939000F894D6
:10046000A9B7A160A9BF84FF02C0A0E4ABBF3FBE93
:1004700018953FB64CB55DB58F7EABB7A074A21191
:100480008061A0E0ABBFA9B7AE7FA9BF789481FD22
:1004900026C096FFA2E096FDA3E0A5BF8260A0B3B0
:1004A00096FDA095A2FF05C040936400509365009F
:1004B00033C196FFA3E096FDA2E0A5BFAA27A064E2
:1004C000AABF8D7FA92FAF7109F417C140E0A0B377
:1004D00096FDA095A2FD11C140938D0004C196FF29
:1004E000A3E096FDA2E0A5BF8D7F61FF6BC096FFE4
:1004F000A2E096FDA3E0A5BFAA27A064AABF8260E0
:100500004093880050938900A09086004A19B090CB
:1005100087005B09BB24A2E0EA2EA22C483CA0E0A5
:100520005A0730F4A0E1BA2EE22CAAE0AA2E27C086
:100530004836A1E05A0730F4A8E0BA2EE22CAFE02A
:10054000AA2E1DC0403DA2E05A0730F4A4E0BA2E06
:10055000E22CAEE1AA2E13C0403AA5E05A0730F4CF
:10056000A2E0BA2EE22CACE3AA2E09C04839A8E0DA
:100570005A0728F4A1E0BA2EE22CA8E7AA2EC42E2E
:10058000A0918A00CA1AD52EA0918B00DA0ADD202C
:100590002AF4AFEFC094D094CA1ADA0A20928C00E1
:1005A000CA14DE0418F4A1E0A0938C0040938A00E2
:1005B00050938B00409188005091890040938600B1
:1005C00050938700A09164004A1BA09165005A0BCC
:1005D00094FD7CC093FD7AC092FD76C056954795F8
:1005E00091FD72C05695479590FD6EC0D52EC42ED4
:1005F000D694C79461FD0CC0AC2DAC51AD2DA2407A
:1006000008F07BC0DD2021F4AC2DA85C08F475C097
:10061000A0E0EA2E97FD08C0E090C200A091B400CF
:10062000A33011F4E090CA00AAEFEA0EF22CF21CFB
:10063000CE18DF084FB74170A091B400A330A9F4E1
:10064000442329F095FD11C0F894906204C095FFF1
:100650000CC0F8949F7D919890989398949A979A4B
:10066000959A71FD01C060687894442369F0A09167
:10067000B400A33031F4AFEFC094D094CA1ADA0AB0
:1006800003C040E050E022C0A091B400A33049F480
:10069000CC0CDD1CA5E0CA1AD20818F4A0E0CA2EC2
:1006A000D22CAFEFCA16D20418F04FEF50E00EC0B4
:1006B000F090A700CF9C412D000C441F50E008F0A3
:1006C00012C04FEF50E00FC05695479594FF07C0FA
:1006D000552309F04FEFA42FA6954A0F521D4F3F07
:1006E000520508F04FEF40938D00816061FF05C017
:1006F000AFE1A095A923AB299A2FA8E1A0936600AA
:10070000A92FAF7119F4AAE0A093660061FD04C09F
:10071000A92FAF7109F08F7EA6E0A0936700A92FE3
:10072000AF7119F4AAE0A0936700F894A9B7A1608B
:10073000A9BF84FF02C0A0E4ABBF3FBE189511E083
:100740000AC013E008C01AE006C01EE104C014E6A7
:1007500002C018EC00C005E1BB27BA95F1F70A9575
:10076000D9F71A95C1F708952AE338E709C020E3BD
:100770003CE806C02AE234EB03C025E238EC00C0B6
:10078000652CB1E05B2E12E095FD9F7D95FF906298
:10079000BB27979ABA95F1F7552009F0909ABA9528
:1007A000F1F79098BA95F1F79798BA95F1F7552027
:1007B00021F095FF919A95FD939AB091A800BA9572
:1007C000F1F795FF919895FD9398B7E8BA95F1F7F1
:1007D0001A95D1F6022FB22FBA95F1F70A95D9F7EB
:1007E0003A9571F6979A562C0895221B39E0001F0E
:1007F0003A9509F40895221F211B18F4210F8894BB
:10080000F6CF0894F4CF622C722CB0E08894B395A4
:10081000221F331FE0F7379527958894912E802E5D
:10082000020B130B10F4192D082D10F4889401C03D
:100830000894661C771CBA9571F7172D062D08953C
:10084000322D11232AF43A9500951095031B130BB2
:10085000F894029F712C002D129F912C802C78947B
:10086000780C172D921C292DB4E06B2E2695179528
:1008700007956A94D9F7332321F000951095031B4F
:10088000130B0895089566FF21C01091740016950A
:10089000009173000795B0917700B01B0B2FB091BA
:1008A0007800B10B1B2F28F40038BFEF1B0740F076
:1008B00009C00F37120508F405C00FE710E002C0A9
:1008C00000E81FEF00937C0010937D00089566FF01
:1008D00039C000917C00B09179000B0F10917D0020
:1008E000B0917A001B1F20E030917D0033230AF481
:1008F0002A95B0917B002B1F1AF4203F40F00AC0CC
:100900002F3008F407C00FEF1FEF2FE003C000E007
:1009100010E020EF30916300B09192003B1718F483
:10092000332331F009C0B0917D00BB235AF004C0DD
:10093000B0917D00BB2332F40093790010937A00CC
:1009400020937B00089566FF2FC02091CD00009179
:100950007C00000F10917D00111F72DF11232AF41B
:100960000038BFEF1B0740F009C00F37120508F42D
:1009700005C00FE710E002C000E81FEF002352F0AF
:10098000B0916200B01B0B2F18F0013008F00AC0C4
:1009900001E008C000950F5FB09162000B0F08F0F6
:1009A00001C00FEF00937E00089566FF2DC02091D7
:1009B000CE0000917A0010917B0042DF11232AF4CF
:1009C0000130BFEF1B0740F009C00F3F120508F4CC
:1009D00005C00FEF10E002C001E01FEF112352F03D
:1009E000B0917E00B01B0B2F18F0013008F00AC048
:1009F00000E008C000950F5FB0917E000B0F08F07B
:100A000001C00FEF0093630008950FEF677FB72FCA
:100A1000B670E9F46860B0917400B83008F0677F90
:100A2000B0917400A1F00FEF10917400DEDEF89425
:100A3000B09170000B9F112D002D7894112309F0B7
:100A40000FEFB09195000B1710F4009195000093F3
:100A5000940008956FC005D374FFB7E074FDB7E04C
:100A6000B068B064B7B9B6B1B068B064B6B967DEA3
:100A700074FFB7E074FDB7E0B068B064B7B9B6B161
:100A8000B068B064B6B9B6B1B6FDFDCF04B115B16A
:100A9000B6B1BF77B6B938D321E02093A30030E0D8
:100AA0003093A400732E7694622E6694620E731EA9
:100AB000262D372D0217130778F08090A300B1E0A0
:100AC000B80DB093A3008090A400B0E0B81DB0931F
:100AD000A400260D371DEECF8090A3009090A400B7
:100AE0001091A40016950091A300079516950795FF
:100AF000B091A300B00FB093A100B091A400B11FBA
:100B0000B093A20023E0169507952A95E1F720916E
:100B1000AF002A9529F42092A3002092A4000AC0D5
:100B20002A9521F0800E911E2A95E1F78092A3006C
:100B30009092A40008952091AF00B6B1B6FDFBCF0E
:100B400004B115B1B6B1BF77B6B9B091A500B395F0
:100B5000B093A500B83060F12092A500B091CC0010
:100B6000BB2321F1112329F0B091A600BF3F61F012
:100B700009C0B091A6000B1739F020F4BB2321F077
:100B8000BA9502C0B395E1F300919200B093A6002C
:100B9000B03050F400ECB03038F400E8B03020F45D
:100BA00000E4B03008F400E0009392007F7E0895E6
:100BB000B0919200B39511F0B0939200B091A5005E
:100BC000B73009F47061089502E3F894B091D00051
:100BD0000B9F012D000C001F7894B09192000B1711
:100BE00010F0009192000093610000936300502E7A
:100BF00000939500089520927300B8E0B0937400BC
:100C000008952091800030918100F8940CB51DB5B5
:100C1000200F311F3BBD2ABD6160B0E1B8BF7894A1
:100C20002091710030917200009371001093720056
:100C3000021B130B2091730030917400622E732EEF
:100C4000B4E08B2EB2E09B2EB0917400B43010F063
:100C50008A949A94B83010F08A949A94769467940F
:100C60008A94E1F726193709992021F016950795FE
:100C70009A94E1F7200F311F209373003093740092
:100C800008F00895BFEFB0937300B0937400089517
:100C90002091820030918300F8940CB51DB5020FAD
:100CA000131F1BBD0ABD6160B0E1B8BF7894089501
:100CB00060FDFECFEDDF0895B091BE0000916E00A3
:100CC000023808F0B395003A08F0B395B63008F052
:100CD000B5E09B2EBCE08B2EB0917400B33030F4A5
:100CE0008394839482FF02C083948394B23030F45F
:100CF0008394839482FF02C08394839471FF03C022
:100D0000B3E09B2E822C109174000091730024E0BC
:100D1000169507952A95E1F70819120928F0B02FC2
:100D2000B250B12FB20910F402E010E0312F202FA1
:100D3000712E602E76946794B92DB330E9F0B0FD32
:100D400005C0060D171D262D372D06C0000F111FDB
:100D50000250120922E030E0B92DB33068F0209340
:100D6000840030938500009380001093810060928E
:100D70008200709283000895009384001093850090
:100D800020938000309381006092820070928300F3
:100D9000089560FDFECF20918200220F30918300E4
:100DA000331FB72FB67021F020917300309174007B
:100DB000F8940CB51DB5020F131F1BBD0ABD616071
:100DC000B0E1B8BF7894089560612092760020E089
:100DD00004C060612092760020E2B72FB67009F05F
:100DE0006F7E789460FD05C0B0917600BB2309F05A
:100DF000089501E063FF0AC0B0917400B33008F0B9
:100E000002E0B0917400B63008F003E071FF01C059
:100E100006E060FD06C0B0917600BB2311F0789427
:100E200008951AE083FF1AE0789400000000F89417
:100E300062FD03C014E183FF14E171FF01C018E7F4
:100E4000B4B530919900B31BB10B18F3B091760093
:100E5000B395B0937600B5E03B2F6B2E722CB8B1F2
:100E6000B072B21709F073943A95C9F77394761477
:100E700088F464FFB2CF6F7E3CB56DB470907300A0
:100E800080907400370D681C6BBC3ABD6160B0E1A6
:100E9000B8BFA3CF64FDA1CF0A9509F0BACF78946B
:100EA000089571FF0AC0B0916D00B395B0936D00C5
:100EB00060FD0CC020926D0009C060FD07C064FD9C
:100EC00005C067FD03C0BF91BF919AC408952091EA
:100ED000840030918500F8940CB51DB5020F131FE6
:100EE0001BBD0ABD6160B0E1B8BF78940895EFDF23
:100EF00000E063FF03C064FF01C001E0F8941091BB
:100F00006E00B7E01B9F212D102D7894200F2695A1
:100F10001795269517952695179510936E001837F7
:100F200018F4B8E7B0936E0000916E00B0916F00B6
:100F30000B1720F0606291989098939860FDFECF17
:100F40000895F894949A979A959A82FF07C0E2E0E0
:100F5000F1E073FF03C0B5E0BA95F1F7B09174000A
:100F6000BC7F81F0552021F095FF919A95FD939AD1
:100F7000B6E0BA95F1F795FF919895FD9398B5E095
:100F8000BA95F1F795FF949895FD9598B2E0B093D6
:100F90007500ABC0F89495FF939895FD919882FFEA
:100FA0000DC0E2EFF0E073FF0BC0979A95FF959AA2
:100FB00095FD949AB5E0BA95F1F702C0ECEAF0E03D
:100FC00062FF03C0552009F0909AB3E0B09375001A
:100FD0008CC0F894949A979A959A82FF07C0E2EE93
:100FE000F0E073FF03C0B5E0BA95F1F7B09174007B
:100FF000BC7F81F0552021F095FF939A95FD919A41
:10100000B6E0BA95F1F795FF939895FD9198B5E004
:10101000BA95F1F795FF959895FD9498B4E0B09343
:10102000750063C0F894909882FF0DC0E2EDF0E087
:1010300073FF0BC095FF949A95FD959A979AB5E02A
:10104000BA95F1F702C0E4EAF0E062FF06C055206D
:1010500021F095FF919A95FD939AB5E0B0937500B4
:1010600044C0F894949A979A959A82FF07C0EFEB40
:10107000F0E073FF03C0B5E0BA95F1F7B0917400EA
:10108000BC7F51F0552009F0909AB6E0BA95F1F77F
:101090009098B5E0BA95F1F79798B6E0B0937500DF
:1010A00024C0F89495FF919895FD939882FF10C005
:1010B000E5E1F1E073FF0EC095FF949A95FD959AD6
:1010C00095FF959A95FD949AB5E0BA95F1F702C00F
:1010D000E4EBF0E062FF06C0552021F095FF939A03
:1010E00095FD919AB1E0B093750067FF0AC00CD0EE
:1010F000B5E0BA95F1F7B5E0BA95F1F794989798FD
:1011000095986F7D7894089523EA30E0F9019198DD
:1011100090989398949A979A959A6B7F0895ACEAD1
:10112000B0E00FEF0D930D930D930D9303E00D932E
:1011300004E00D930AE00D9303E00D9301E00D939D
:1011400001E00D93A8EBB0E001E00D930FEF0D93DC
:101150000D930FEF0D930D930D9303E00D9306E0A8
:101160000D930FEF0D930D9305E20D9300ED0D938D
:101170000AEF0D930AEF0D9304E00D930DE00D932C
:1011800001E00D9300E00D930AE70D930FEF0D932F
:1011900001E00D9308952091BF0009E011E0223095
:1011A00011F405E011E0233011F405E012E02430E1
:1011B00011F405E013E0253011F409E017E02630C2
:1011C00011F400E010E000939F001093A000209124
:1011D000B3008B7F233009F48460777F233009F4D8
:1011E0007860B091B400B33019F09F7DB1FD90628A
:1011F0009F7BB091B500B1FD9064B22FB23011F079
:10120000886001C0877F0895ECE1F0E00091AC00B8
:101210000A95E00FF21DB491B093CD000091AD009E
:101220000A95E00FF21DB491B093CE006DDF0895E2
:10123000EAE2F0E00091C7000A95E00FF21DB491D8
:10124000B093CF0061DF0895E8E3F0E00091B200D1
:101250000A95E00FF21DB491B093D00055DF0895C8
:101260000895B091C8000FEF1CE0B23011F400EA0D
:101270001AE0B33011F402E815E000936F00109308
:101280007000089508952091C2003091C30097FF27
:1012900002C020E03FEFB32FB21B6B2EB25810F408
:1012A000B2E86B2E00E00395609EB12DB058D8F3E4
:1012B0000093A7000895F894E3E0F0E0B9E0B7BF29
:1012C000B491B078C1F3F894A895B1B5B861B1BD47
:1012D000B0E0B1BDB4E0BEBFBFE5BDBF15DFB0E05B
:1012E000B8BBB0E1B7BBB0E0B5BBB0E0B4BBB0EBEE
:1012F000B2BBBBEBB1BB2224A0E0B0E02D92AA317F
:10130000E9F7A0E6B0E00FEF2D920A95E9F707DFC5
:1013100097D241DF79DF8CDF97DFA2DFA2DFB2DF78
:10132000B2DF0091C4000093A800EEDEB2E0B3BFCC
:10133000B2E0BEBDB2E0B5BDF8940BDA15DA05DA5D
:1013400016DA03DA17DA01DA06D303DA02DAFFD99A
:10135000B1E5B8BFB9BFB0B7B860B0BFB6B1B4609F
:10136000B6B9EDD9789476DBB0E4BBBFBB27B064E7
:10137000BABF8D7FEED9B1E0B0936900626025E01D
:10138000B0918C00BB2309F425E0DBD9B0918D002E
:10139000B230A8F3B92FBF7100918F0000938E0077
:1013A000B0938F00B01759F72A9551F76D7F96FFCC
:1013B000B3E096FDB2E0B5BFBB27B064BABF8D7F86
:1013C000C6D9BFD902E0B92FBF7109F400E0B091CE
:1013D0008D00B017B0F3F894C7D9C6D9C5D97894A1
:1013E000B8D920927F00B091B400B33009F472C034
:1013F000A8D9B091B800B13008F46CC0B0916900C0
:10140000B13008F467C0B92FBF71C1F0B0918D0041
:10141000BF3F08F45FC0F894B0D9789498D9B091E0
:101420008D00B130C0F7F8949FD98DD99DD97894AB
:101430008ED9B0918D00BF3FB0F3BFC2B8E09B2EF4
:101440009068F89420DF789482D9F8949F771BDF16
:1014500080908D00B0918D00BF37789408F442C021
:101460006ED9F8948AD978949A9451F7B82DB550DA
:10147000B093C3006ED9F89410D272D27894BAE0C7
:101480009B2E9068F894FFDE789461D9F8949F774A
:10149000FADE80908D00B0918D00BF37789478F798
:1014A0004ED9F89461D94FD95FD978949A9449F775
:1014B000B82DBB5FB093C2004CD9F894EED15FD287
:1014C000789445D9F894DFDE7894B0918D00BF3FD1
:1014D000C0F373C200918D00B0917F000B1710F024
:1014E00000937F0034D901E0B091B400B35009F407
:1014F00005E0B0918D00B01708F075CFF8943DD994
:101500003CD93BD9789425D92092690020926A0071
:1015100020926B00B0916A00B395B0936A00BF3F10
:1015200069F5B0916B00B395B0936B00B091C600B4
:1015300009E1BA9559F002E3BA9541F00DE7BA9581
:1015400029F00AEFBA9511F020926B00B0916B0070
:10155000B017A0F0B0916B00BA95B0936B00B4EBEC
:10156000B0936A00B091C500B093A800F89405D973
:101570007894B091C400B093A800E9D8E4D8B091B1
:101580006600BB2321F4B92FBF7109F4F7CEB091E7
:101590008D00B63008F4BECFB091B400B35009F05E
:1015A000D6D8B0916600BB2309F4E8CEF894ACDD40
:1015B000209261002092620020926300522C789465
:1015C000B091B100B09396002092770020927800FD
:1015D0002092790020927A0020927B002092A50030
:1015E00060E070E020926E0006DBB8E0B093A500EA
:1015F0007061A5D874FFB7E074FDB7E0B068B0645F
:10160000B7B9B6B1B068B064B6B9B6B1B6FDFDCF82
:1016100004B115B1B6B1BF77B6B9112309F00FEF18
:101620000093A60088DAB8E0B093A50070618090BE
:10163000B300B2E0B093B300AEDD8092B300F89493
:10164000BFEFB0939200C0DAB0916100B093920006
:10165000B0939300B09394007894B1E0B09361009C
:10166000B09363005B2EB0939B00B0919100B09358
:101670009A007160726020926D00F3DC12DDC1DAB5
:10168000BADA1ADB04C087DD2092A5007F7E95FFC1
:10169000B2E095FDB4E0B068B064B7B99ADB01DCA4
:1016A00016DCF0D824DC4DDCACDA02DB05DB71DBC8
:1016B000B3E0B068B064B7B987DBF3DB08DCE3D82C
:1016C000A4D915DC67DC9DDAF3DAF6DA62DB95FF84
:1016D000B4E095FDB2E0B068B064B7B97ADBE1DBA5
:1016E000F6DBF5D804DC75DC8CDAE2DAE5DA51DB1E
:1016F00095FFB2E095FDB4E0B068B064B7B964DBC3
:10170000D0DBE5DB20D9F3DB8DDC7BDAD1DAD4DA90
:1017100040DBB3E0B068B064B7B95BDBC2DBD7DBFA
:1017200044D9E5DB9EDC6DDAC3DAC6DA32DB95FF3D
:10173000B4E095FDB2E0B068B064B7B945DB74FFC2
:10174000B7E074FDB7E0B068B064B7B9B6B1B068DF
:10175000B064B6B9A6DBBBDBCADBA3DC52DAA8DA1D
:10176000ABDAE9D916DB71FF25C067FD23C0B09164
:101770009500B0939200B0939300B0919100B09314
:101780009A00B1E0B0939B0014E624E1B0916D00A3
:10179000B11750F07D7F746020936C00BFEFB09361
:1017A0009200B093930006C0B0918D00B13008F064
:1017B0006ECF26C072FF10C067FD0EC0B0916C00E6
:1017C000BA9511F47B7F5FCFB0936C00B0918D0020
:1017D000B13008F05CCF14C0B0919000B23880F402
:1017E000B92FBF7121F4B0916600BB2349F0B091CD
:1017F000740000EF67FF01C000E6B01708F447CFA0
:10180000F89482DC8090B300B2E0B093B300C3DC04
:101810008092B300209261002092620020926300C7
:10182000522C209296007E7F789489D76DDCB92F58
:10183000BF7129F4B0916600BB2309F49FCD66CE39
:10184000EDE0F0E023D00A3509F01BC0EEE0F0E057
:101850001DD0053A09F015C03AE0ACEAB0E0E3E08B
:10186000F0E014D00D9331963A95D9F735E1A8EB15
:10187000B0E0EFE0F0E00AD00D9331963A95D9F759
:1018800002C04DDC0AD0E4E2F0E00895E199FECF19
:10189000EEBBFFBBE09A0DB308951ED03AE0ACEA70
:1018A000B0E0E3E0F0E00D910FD031963A95D9F732
:1018B00035E1A8EBB0E0EFE0F0E00D9105D0319616
:1018C0003A95D9F712D00895E199FECF0DBBEEBB42
:1018D000FFBBE29AE19A0895EDE0F0E00FEFF4DF4C
:1018E000EEE0F0E00FEFF0DF0895EDE0F0E00AE564
:1018F000EBDFEEE0F0E005EAE7DF08953091A900C4
:101900000091AA00313011F40093B000323011F48C
:101910000093B100333011F40093B200343011F46D
:101920000093BE00353011F40093C700363011F437
:101930000093BF00373011F40093B300383011F436
:101940000093C800393011F40093B4003A3011F418
:101950000093B500089525E0FCD62A95E9F708958F
:1019600003D705D707D709D7EED6FED600D702D7BB
:1019700004D7E9D6F9D6FBD6FDD6FFD60895FDD615
:10198000F9D6F5D6F1D6DFD6F8D6F4D6F0D6ECD621
:10199000DAD6F3D6EFD6EBD6E7D608958090A90035
:1019A0009090AA00E1D6E0D6DFD6CDD68A94D1F7C2
:1019B000E4D6C9D69A94E1F70895F894D1DF7894E3
:1019C000CADFC9DFB1E0B093A900B1E0B093AA00CB
:1019D0002092AB00F894E2DF7894B5E06B2E709023
:1019E0008D00B7D6B0918D007B16C9F7B13018F0D5
:1019F000BF3F40F107C082DFF8944FDFB1DFB8E0AE
:101A0000B1BDA9DF6A9459F7B091AB00B395B0931B
:101A1000AB00B33008F4DECF9EDFB091AA00B395DF
:101A2000B093AA00F894B091A900BA95E6E4F0E06A
:101A3000EB0FF21D049178940395B091AA00B017B2
:101A400008F4C6CF88DF87DFB091A900B395B093C3
:101A5000A900B091A900BB3008F4B7CF60DBF894BF
:081A60001CDFB8E0B1BD77DF27
:00000001FF
